:100000000C94ED020C9434030C9434030C943403DC
:100010000C9434030C9434030C9434030C94340384
:100020000C9434030C9434030C947D0C0C944F0DFD
:100030000C9434030C9434030C9434030C94340364
:100040000C9434030C94C3210C9434030C943403A7
:100050000C9434030C94551B0C9434030C9434030B
:100060000C9434030C9434030C9434030C94340334
:100070000C9434030C9434030C9434030C94340324
:100080000C9434030C9434030C9434030C94340314
:100090000C9434030C9434030C9434030C94340304
:1000A0000C9434030C9434030C943403BC0DDE0D17
:1000B000D10EDE0DD10E230E460ED10E9B0EAE0ECE
:1000C00098119811C711C7110A12441251145114F2
:1000D0005D125114521352132514511451143C142F
:1000E000014702477432014702477432012102215D
:1000F0007432012802280001470247743201470286
:10010000477432012002207432012802280001477E
:1001100002477432014702477432011F021F7432D2
:100120000128022800014702477432014702477440
:1001300032011E021E74320128022800000001C094
:1001400002C003C004C005C0018C028C2E004C000C
:100150002900E100358200001E00140004001D008B
:1001600034004D821F001A0015001B00E1042A71A3
:10017000200009001600060050002C722100130018
:10018000170019004F004A0022000A00070005006E
:100190000000E2005000025400002E000000012088
:1001A0004F00025400002D000000E20023000D006B
:1001B0000B000E000000E60024000F0011001000EC
:1001C00052004B002500180008003600510028722C
:1001D00026001C000C0037002F002B712700330075
:1001E0001200387130004E832D0031003400E500DC
:1001F000008200002E004C002900E1003582000042
:100200001E00140004001D0034004D821F001A005F
:1002100016001B00E1042A712000080007000600F8
:1002200050002C7221001500090019004F004A00EF
:10023000220017000A0005000000E20050000254EE
:1002400000002E00000001204F00025400002D008D
:100250000000E20023001C000B0011000000E6007B
:10026000240018000D00100052004B0025000C0067
:100270000E00360051002872260012000F003700D1
:100280002F002B71270013003300387130004E838C
:100290002D0031003400E500008200000100010063
:1002A00001000100010000003A001E0220022202AB
:1002B000010001003B001F02210223020100010096
:1002C0003C002F0226022F00010001003D003002F9
:1002D00027023000010001003E00310235003502E6
:1002E0000000010001000100000001000000010009
:1002F0000100010000000100000001003F00520069
:1003000051002402000001004000240021001E00D2
:10031000010001004100250022001F0037000100FC
:100320004200260023002000270001004300250290
:100330002E0231002E0001004400450001000100A2
:1003400001000000000000000000000000000000AC
:10035000000006200220000000000100000007202D
:100360000320000000000100000000000420000045
:100370000000010000000000052000000000010056
:10038000000000000000000000000100000000006C
:10039000000000000000010000000000000000005C
:1003A000000001000000000000000000000001004B
:1003B000000000000000000000000100000000003C
:1003C000000000000000010000000000000000002C
:1003D000000001000000000000000000000001001B
:1003E00000000000000000000000000016034500AF
:1003F000720067006F0044006F0078002000450025
:100400005A00000016034500720067006F004400A8
:100410006F007800200045005A0000000403090422
:1004200009026D00040100A0FA09040000010301A3
:100430000100092111010001223F00070581030885
:10044000000A090401000103010200092111010051
:1004500001224D000705820308000A090402000179
:100460000300000009211101000122360007058365
:100470000308000A09040300010300000009211118
:100480000100012239000705840310000112011048
:100490000100000008EDFE07130100010200010544
:1004A000010906A101050719E029E71500250195B5
:1004B0000875018102050819012905950575019145
:1004C000029501750391010507190029771500258B
:1004D00001957875018102C005010980A10185029D
:1004E00016010026B7001A01002AB7007510950101
:1004F0008100C0050C0901A1018503160100269C9D
:10050000021A01002A9C02751095018100C00501A4
:100510000902A1010901A100050919012905150018
:10052000250195057501810295017503810105017C
:10053000093009311581257F950275088106093832
:100540001581257F950175088106050C0A3802156D
:1005500081257F950175088106C0C005010906A1A6
:1005600001050719E029E7150025019508750181A6
:100570000295017508810105081901290595057580
:100580000191029501750391010507190029FF15D5
:100590000025FF950675088100C0000000000000DE
:1005A0000000000000010204060A0F17202C3A4A3E
:1005B0005D71879DB3C7DAE9F5FCFFFCF5E9DAC7A1
:1005C000B39D87715D4A3A2C20170F0A0604020179
:1005D0000000000000000000000011241FBECFEF4B
:1005E000DAE0DEBFCDBF04B603FE27C08091ED0187
:1005F0009091EE01A091EF01B091F0018730904B06
:10060000A740B04BD1F41092ED011092EE01109280
:10061000EF011092F00114BE84B7877F84BF0FB63C
:10062000F894A89580916000886180936000109292
:1006300060000FBEE0E0FFE3099511E0A0E0B1E04B
:10064000E8E2F7E402C005900D92A433B107D9F7B0
:1006500021E0A4E3B1E001C01D92AD3EB207E1F795
:100660000E94C4090C9492230C940000FC01623097
:1006700021F128F4662349F0613071F036C064300E
:1006800041F108F1653059F130C08281882311F0C1
:1006900085EE0CC085EE0EC08281882351F085EE78
:1006A0000E94321085EE0E94FA1083EE0E943210F2
:1006B0001CC083EE0E94FA1018C08281811115C0FF
:1006C00085E291E00895828181110FC08EE091E072
:1006D00008958281811109C087EF90E00895828199
:1006E000811103C080EE90E0089580E090E00895CD
:1006F00008956091B1017091B2018091B301909120
:10070000B4010E94821A56985E9825982D982698D2
:100710002E9827982F98823019F0833021F0089571
:10072000259A2D9A0895269A2E9A08950C94790365
:1007300056985E9825982D9826982E9827982F9849
:100740008FEF90E0909389008093880090938B00C6
:1007500080938A0090938D0080938C00259A2D9A27
:100760002FEF80E792E0215080409040E1F700C0F9
:100770000000269A2E9A2FEF80E792E021508040C9
:100780009040E1F700C00000279A2F9A2FEF80E7F2
:1007900092E0215080409040E1F700C00000259891
:1007A0002D982FEF80E792E0215080409040E1F7B4
:1007B00000C0000026982E982FEF80E792E021508D
:1007C00080409040E1F700C0000027982F9856988D
:1007D0005E9825982D9826982E9827982F980895FA
:1007E00089EA8093800089E08093810024982C9886
:1007F0003F988AB18F748AB96E98479A8BB1806B93
:100800008BB9769A0E9498030C94780380E28093C7
:1008100000018091340181110EC00E94550481E0D5
:10082000809334012FEF83ED90E32150804090407E
:10083000E1F700C0000080E40E945B0480930001A7
:1008400081112EC00E94850480930001811128C06F
:100850000E94850480930001811122C08FE30E94D1
:1008600085048093000181111BC00E947D0480E4F7
:100870000E945B0480930001811112C08CE00E94F1
:1008800085048093000181110BC00E948504809330
:100890000001811105C08FE30E948504809300014F
:1008A0000E947D048091000108951092B9008AE0B1
:1008B0008093B800089594EA9093BC009091BC0096
:1008C00097FFFCCF9091B900987F983021F090313C
:1008D00011F081E008958093BB0084E88093BC0010
:1008E0008091BC0087FFFCCF8091B900887F883160
:1008F00011F0803471F780E0089584E98093BC00A2
:100900008091BC0084FDFCCF08958093BB0084E8F7
:100910008093BC008091BC0087FFFCCF9091B90010
:10092000987F81E0983209F480E0089584E880930C
:10093000BC008091BC0087FFFCCF8091BB00089574
:1009400080910001811115C080E40E945B048093B6
:10095000000181110CC082E10E9485048093000196
:10096000811105C08FEF0E948504809300010E94D1
:100970007D0484B1807F84B985B1807F85B98AB1D7
:10098000837F8AB98BB1837F8BB93E98469808954F
:100990000E940604809300010E94A00480B38C7022
:1009A00080BB81B3836F81BBE4E4F1E0A6E3B1E0F7
:1009B00011921D9281E0E235F807D1F70C94F00313
:1009C0009F92AF92BF92CF92DF92EF92FF920F93DE
:1009D0001F93CF93DF9380910001882379F080915A
:1009E00035018F5F80933501811108C00E94060494
:1009F00080930001811102C00E94980386E3E82ED3
:100A000081E0F82E8701C0E0D0E0BB24B39492E0EF
:100A1000A92ECC24C394D12CC730D10500F58091E8
:100A20000001811164C080E40E945B048093000196
:100A3000811112C082E10E9485048093000181111E
:100A40000BC0C6010C2E01C0880F0A94EAF78095EE
:100A50000E948504809300010E947D0448C0CA3032
:100A6000A1F028F4C83059F0C93061F005C0CC308D
:100A700089F070F0CD3089F0209A289810C0219A22
:100A800029980DC0229A2A980AC0239A2B9807C049
:100A9000529A01C0539A5B9802C03E9A4698E0EA87
:100AA000EA95F1F78FB181708B25799902C032E018
:100AB00001C030E0832B7C9902C034E001C030E0FB
:100AC000832B7D9902C028E001C020E0822B7E9913
:100AD00002C090E101C090E0892B9FB19095991FD1
:100AE0009927991F9295990F907E892B0FC080911D
:100AF000000181114AC080E40E945B0480930001E0
:100B0000882381F1912C0E947D04892DD8019C912C
:100B1000981719F08C93A09201010E94A0042196CD
:100B20000F5F1F4FCE30D10509F076CF80910101C4
:100B3000882369F1815080930101882339F0EFE91E
:100B4000FFE03197F1F700C0000021C0E4E4F1E0DC
:100B5000D7018D917D018193B4E4EB16B1E0FB06E2
:100B6000B9F715C083E10E948504809300018111CB
:100B7000C9CF81E40E945B04809300018111C2CF40
:100B80000E949604982E9094BECF80E0BFCF0E9422
:100B9000960381E0DF91CF911F910F91FF90EF902D
:100BA000DF90CF90BF90AF909F900895E82FF0E036
:100BB000EC5BFE4F8081089508958B3B910580F496
:100BC000883A910548F5853A9105D8F48430910525
:100BD00008F0B2C0019709F06EC081E090E008957E
:100BE000803E910508F467C0883E910508F4A4C0D2
:100BF0009C01205F31092031310508F05CC090650F
:100C00000895853A910509F459C0863A910509F08D
:100C100058C082E890E40895883A910509F454C0D8
:100C2000893A910509F453C08A3A910509F452C0F2
:100C30008B3A910509F451C08C3A910509F450C0E2
:100C40008D3A910509F44FC0803B910509F44EC0DF
:100C50008E3A910509F44DC08F3A910509F44CC0C4
:100C6000813B910509F44BC0823B910509F44AC0D0
:100C7000833B910509F449C0843B910509F448C0C0
:100C8000853B910509F447C0863B910509F446C0B0
:100C9000873B910509F445C0883B910509F444C0A0
:100CA000893B910509F443C08A3B910509F442C090
:100CB00080E094E4089580E090E0089581E890E475
:100CC000089583E890E4089582EE94E4089589EE0F
:100CD00094E408958AEE94E4089585EB94E40895ED
:100CE00086EB94E4089587EB94E408958CEC94E407
:100CF00008958DEC94E4089583E895E408958AE8D6
:100D000095E4089582E995E4089584E995E40895C9
:100D100081E296E4089583E296E4089584E296E4FD
:100D2000089585E296E4089586E296E4089587E2C0
:100D300096E408958AE296E40895089524E5829F52
:100D4000C0011124FC0126E0729FE00DF11D112469
:100D5000E60FF11DEE0FFF1FE45BFE4F85919491AE
:100D60000895880F991FFC01E454F04085919491F7
:100D70000895880F991FFC01E45CFE4F85919491C2
:100D8000089524E5829FC0011124FC0146E0749F70
:100D9000E00DF11D1124E60FF11DEE0FFF1FE45BC6
:100DA000FE4F859194919C013A9521154FE13407AE
:100DB00008F425C13F512115304120F49F700E9455
:100DC000B90608959C0130532115304118F4992734
:100DD000906C0895811520E5920769F40E947314C0
:100DE0004FEF84E39CE0415080409040E1F700C029
:100DF00000000C947A1B813020E5920731F4809139
:100E0000CC0181608093CC0108959C01305521155F
:100E1000304108F05CC0292F33272F703327213051
:100E20003105E9F4AC0164E0440F551F6A95E1F720
:100E300044275370BC016370772702C0220F331F11
:100E40006A95E2F73C68242B352B73E0880F991FD5
:100E50007A95E1F780769927822B932B089522309B
:100E6000310529F4982F8827816F906A08952330DF
:100E70003105A1F4AC0133E0440F551F3A95E1F779
:100E8000407E57708370992721E030E002C0220F26
:100E9000331F8A95E2F7C9019C6816C024303105DA
:100EA00031F5AC0123E0440F551F2A95E1F7407E50
:100EB00057708370992721E030E002C0220F331F62
:100EC0008A95E2F7C9019A68842B952B08959C01B5
:100ED00030572115304118F49F70906208959C019D
:100EE00030582115304118F49F70906A0895803E63
:100EF0009105E0F4803C910558F58133910509F4A2
:100F00006FC048F48932910509F463C08A329105B3
:100F100009F46DC072C089339105E9F082389105FA
:100F2000D1F08533910509F44DC067C0833E91052A
:100F300081F138F4803E9105B9F0823E9105D9F0F7
:100F40005CC0863E910561F1873E9105A1F155C0D7
:100F50000E94B10608952091DE0120FD02C021FF0C
:100F60004CC080EE90E049C08091DE0180FFF9CF57
:100F700089E390E042C08091DE0182FF0EC0809143
:100F8000DE0184FF03C080E090E037C083EE90E094
:100F900034C08091DE0182FFF2CF82EE90E02DC05E
:100FA0008091DE0183FF0BC08091DE0184FDEBCFD9
:100FB00087EE90E022C08091DE0183FFF5CF86EEC0
:100FC00090E01BC08091DE0185FF07C089E290E0C0
:100FD00014C08091DE0185FFF9CF85E390E00DC05C
:100FE0008091DE0186FF07C08AE290E006C0809112
:100FF000DE0186FFF9CF81E390E00E94DD050895D0
:101000000895809162010895CF93DF9300D01F92DD
:10101000CDB7DEB79C018091E401843019F593E0EF
:1010200099833B832A839093E9008FEF9091E800A6
:10103000815095FD06C095ED9A95F1F7000081115C
:10104000F5CF8091E80085FF0DC040E050E063E0FF
:1010500070E0CE0101960E94710A8091E8008E77BF
:101060008093E8000F900F900F90DF91CF9108953B
:10107000CF93DF9300D01F92CDB7DEB72091E4016C
:10108000243021F522E029839B838A8383E08093A7
:10109000E9008FEF9091E800815095FD06C095ED35
:1010A0009A95F1F700008111F5CF8091E80085FF56
:1010B0000DC040E050E063E070E0CE0101960E9478
:1010C000710A8091E8008E778093E8000F900F906E
:1010D0000F90DF91CF9108959C018091E4018430BD
:1010E000F9F482E08093E9009FEF8091E80091504D
:1010F00085FD06C085ED8A95F1F700009111F5CFC9
:101100008091E80085FF0CC040E050E065E070E0B1
:10111000C9010E94710A8091E8008E778093E800EF
:101120000895CF93DF93EC018091E401843009F0BE
:1011300046C090910C019923D9F090910D0199230B
:10114000B9F08093E9008FEF9091E800815095FD10
:1011500006C095E19A95F1F700008111F5CF8091D5
:10116000E80085FF2CC040E050E060E170E017C06F
:1011700081E08093E9008FEF9091E800815095FD28
:1011800006C095ED9A95F1F700008111F5CF809199
:10119000E80085FF14C040E050E068E070E0CE0158
:1011A0000E94710A8091E8008E778093E80080E1C8
:1011B000FE01A2E5B1E001900D928A95E1F7DF9181
:1011C000CF9108958091E301811109C00E94020C22
:1011D0000E945F0C8091E20084608093E200089599
:1011E0001092E301089508950C94B0210E94101B01
:1011F0000E94B6210E940A0F0C94000842E061ECA4
:1012000081E00E947B0B42E061EC82E00E947B0B5C
:1012100042E061EC83E00E947B0B42E161EC84E000
:101220000C947B0B8091E601833009F455C030F4B7
:10123000813071F0823009F48EC008958A3009F44B
:101240007AC08B3009F460C0893009F09CC020C09E
:101250008091E501813A09F096C08091E800877F8E
:101260008093E8008091E9019091EA01892B21F4B3
:1012700060E182E591E003C060E080E090E070E032
:101280000E94BC0A8091E8008B778093E800089563
:101290008091E501813209F076C08091E901909159
:1012A000EA01009719F0039709F06DC08091E800FA
:1012B000877F8093E8008091E80082FD05C08091DF
:1012C000E4018111F8CF5FC08091F1008093620149
:1012D0008091E8008B7753C08091E501813A09F055
:1012E00052C08091E9019091EA01892B09F04BC02D
:1012F0008091E800877F8093E8008091E80080FF7C
:10130000FCCF80910C0136C08091E5018132D9F586
:101310008091E9019091EA01892BA9F58091E8007B
:10132000877F8093E8000E94B00B8091E701809353
:101330000C010C9473148091E501813221F58091A8
:10134000E800877F8093E8000E94B00B8091E8015D
:101350008093630108958091E501813AA1F4809121
:10136000E800877F8093E8008091E80080FFFCCF51
:10137000809163018093F1008091E8008E778093E3
:10138000E8000C94B00B089584B7877F84BF0FB634
:10139000F894A89580916000886180936000109215
:1013A00060000FBE90E080E80FB6F8948093610073
:1013B000909361000FBE0E94590F0E94020C0E9480
:1013C0005F0C8091E20084608093E20078940E9438
:1013D000EA0E0E945B0F82E091E00E94050F0E94DE
:1013E0009E218091E401853069F40E94D21A809197
:1013F000E2018823B1F30E94FC1A882391F30E9432
:101400005B0AEFCF0E94610FECCF292F33272330E7
:101410003105C9F060F42130310581F02230310509
:1014200009F041C08DE690E020E234E040C0213276
:101430003105E1F02232310531F135C082E190E031
:101440002DE834E034C099278130910549F028F027
:10145000029749F5ECEEF3E005C0ECE1F4E002C0E0
:10146000E4E0F4E0849190E09F0121C06430D8F47E
:10147000E62FF0E0EE0FFF1FEE5DFE4F2081318181
:1014800089E090E014C0643070F470E0FB01EE0F6E
:10149000FF1FE65EFE4F20813181FB01EA5EFE4FB9
:1014A000808190E004C080E090E020E030E0FA012C
:1014B00031832083089580E189BD82E189BD09B42B
:1014C00000FEFDCF8091D8008F7D8093D800809161
:1014D000E00082608093E0008091E00081FDFCCF1D
:1014E0000895CF92DF92EF92FF920F931F93CF93C5
:1014F000DF93EC018B016A010E94CF0B811133C095
:10150000C114D10439F0F60180819181081B190BB7
:10151000C80FD91FE12CF12C0115110519F180918B
:10152000E80085FD16C08091E8008E778093E80082
:10153000C114D10449F0F60180819181E80EF91EB1
:10154000F182E08285E00FC00E94CF0B882321F357
:101550000AC089918093F10001501109FFEFEF1A41
:10156000FF0ADACF80E0DF91CF911F910F91FF90BA
:10157000EF90DF90CF9008952091EB013091EC0136
:101580002617370748F06115710539F42091E800F6
:101590002E772093E80001C0B901FC0120E061151D
:1015A000710579F18091E4018823F1F18530F1F141
:1015B0008091E80083FD3CC08091E80082FD2EC050
:1015C0008091E80080FFEBCF2091F3008091F20042
:1015D00090E0922B6115710551F08830910538F437
:1015E00021912093F100615071090196F3CF21E020
:1015F000089709F020E08091E8008E778093E8005A
:10160000CECF2111CFCF0AC08091E401882361F0B1
:10161000853061F08091E80083FD0AC08091E80088
:1016200082FFF2CF80E0089582E0089583E008957C
:1016300081E008952091EB013091EC0126173707E6
:1016400048F06115710539F42091E8002E77209358
:10165000E80001C0B901FC0120E06115710591F1BC
:101660008091E401882309F440C0853009F43FC02B
:101670008091E80083FD3DC08091E80082FD2FC08D
:101680008091E80080FFE9CF2091F3008091F20083
:1016900090E0922B6115710559F08830910540F466
:1016A00024912093F1003196615071090196F2CF97
:1016B00021E0089709F020E08091E8008E77809380
:1016C000E800CBCF2111CCCF0AC08091E401882360
:1016D00061F0853061F08091E80083FD0AC080915F
:1016E000E80082FFF2CF80E0089582E0089583E071
:1016F000089581E00895982F973068F59093E90058
:10170000981739F07091EC002091ED005091F000A5
:1017100003C0242F762F50E021FD02C09F5FECCF45
:101720003091EB003E7F3093EB003091ED003D7F38
:101730003093ED003091EB0031603093EB0070930B
:10174000EC002093ED005093F0002091EE0027FD77
:10175000E5CF80E008958F708093E90081E00895DF
:101760008091E50187FF11C08091E80082FD05C0EE
:101770008091E4018111F8CF11C08091E8008B774E
:101780000BC08091E401882349F08091E80080FF3C
:10179000F8CF8091E8008E778093E800089520913B
:1017A000E4003091E50095E64091EC00842F8170D3
:1017B00040FF23C08091E80080FD1DC08091E401BE
:1017C000882399F0853099F08091EB0085FD11C058
:1017D0004091E4005091E5002417350729F391501A
:1017E00011F09A01E1CF84E0089582E0089583E04A
:1017F000089581E0089580E008954091E80042FF57
:10180000DDCF08950E94700C0E94780CE0EEF0E0AD
:10181000808181608083E8EDF0E080818F77808334
:1018200019BCA7EDB0E08C918E7F8C9380818F7E68
:1018300080831092E30108950F931F93CF93DF935A
:101840000E94700C0E94780CC8EDD0E088818F77E0
:10185000888388818068888388818F7D888319BC8C
:101860001092E4011092E0011092E2011092E10165
:1018700000EE10E0F80180818B7F80838881816099
:10188000888342E060E080E00E947B0BE1EEF0E0C4
:1018900080818E7F8083E2EEF0E0808181608083B2
:1018A000808188608083F80180818E7F8083888139
:1018B00080618883DF91CF911F910F910895E8EDAA
:1018C000F0E080818F7E8083E7EDF0E080818160B1
:1018D000808384E082BF81E08093E3010C941C0C40
:1018E000E8EDF0E080818E7F80831092E200089521
:1018F0001092DA001092E10008951F920F920FB635
:101900000F9211242F933F934F935F936F937F9385
:101910008F939F93AF93BF93EF93FF938091E100D9
:1019200082FF0BC08091E20082FF07C08091E1003E
:101930008B7F8093E1000E94E90E8091DA0080FFA6
:101940001FC08091D80080FF1BC08091DA008E7F7D
:101950008093DA008091D90080FF0DC080E189BDBD
:1019600082E189BD09B400FEFDCF81E08093E401EE
:101970000E94E20805C019BC1092E4010E94F00820
:101980008091E10080FF19C08091E20080FF15C0C6
:101990008091E2008E7F8093E2008091E20080617E
:1019A0008093E2008091D80080628093D80019BCB7
:1019B00085E08093E4010E94F4088091E10084FFB7
:1019C00030C08091E20084FF2CC080E189BD82E1BB
:1019D00089BD09B400FEFDCF8091D8008F7D809332
:1019E000D8008091E1008F7E8093E1008091E20039
:1019F0008F7E8093E2008091E20081608093E2001C
:101A00008091E001882311F084E007C08091E30019
:101A100087FD02C081E001C083E08093E4010E9461
:101A2000F6088091E10083FF29C08091E20083FFE6
:101A300025C08091E100877F8093E10082E0809360
:101A4000E4011092E0018091E1008E7F8093E1003B
:101A50008091E2008E7F8093E2008091E2008061BD
:101A60008093E20042E060E080E00E947B0B809186
:101A7000F00088608093F0000E94F308FF91EF91DE
:101A8000BF91AF919F918F917F916F915F914F9196
:101A90003F912F910F900FBE0F901F9018951F929E
:101AA0000F920FB60F9211242F933F934F935F9392
:101AB0006F937F938F939F93AF93BF93CF93DF9356
:101AC000EF93FF93C091E900CF708091EC00D82F85
:101AD000D17080FDD0E81092E9008091F000877FFE
:101AE0008093F00078940E94930D1092E900809109
:101AF000F00088608093F000CD2BCF70C093E90098
:101B0000FF91EF91DF91CF91BF91AF919F918F9115
:101B10007F916F915F914F913F912F910F900FBEE9
:101B20000F901F9018951F93CF93DF93CDB7DEB71B
:101B3000AA970FB6F894DEBF0FBECDBFE5EEF1E079
:101B40008091F100819321E0ED3EF207C9F70E94F8
:101B500012098091E80083FF24C18091E5019091F2
:101B6000E601492F50E04A30510508F01AC1FA0148
:101B7000EA5AFF4F0C944723803881F0823809F0ED
:101B800010C18091E9018F708093E9008091EB0092
:101B900085FB882780F91092E90006C08091E10159
:101BA0009091E201911182609091E800977F90936B
:101BB000E8008093F1001092F100C8C0282F2D7F1B
:101BC00009F0EFC0882319F0823061F0EAC08091FB
:101BD000E701813009F0E5C0933009F080E080939F
:101BE000E2012BC08091E701811127C08091E901BA
:101BF0008F7009F4D6C08093E9002091EB0020FF9C
:101C00001CC0933021F48091EB00806214C090914D
:101C1000EB0090619093EB0021E030E0A90102C05D
:101C2000440F551F8A95E2F74093EA001092EA00AC
:101C30008091EB0088608093EB001092E900809126
:101C4000E800877F86C08111ACC01091E7011F7743
:101C50008091E3008078812B8093E3008091E800FD
:101C6000877F8093E8000E94B00B8091E80080FF9E
:101C7000FCCF8091E30080688093E300111102C0E3
:101C800082E001C083E08093E4018BC08058823001
:101C900008F087C08091E7019091E8018C3D53E006
:101CA000950779F583E08A838AE289834FB7F894B0
:101CB000DE01139620E03EE051E2E32FF0E0509386
:101CC0005700E49120FF03C0E295EF703F5FEF7093
:101CD0008E2F90E0EA3010F0C79601C0C0968D9329
:101CE0009D932F5F243149F74FBF8091E800877F94
:101CF0008093E8006AE270E0CE0101960E94BC0A7F
:101D000014C0AE014F5F5F4F6091E9010E94050A68
:101D1000BC01892B09F445C09091E800977F90930E
:101D2000E80089819A810E941A0B8091E8008B77E4
:101D30008093E80036C08038A1F58091E800877F65
:101D40008093E8008091E0018093F1008091E800A9
:101D50008E778093E8000E94B00B23C0811121C0D0
:101D60008091E7019091E80199270297D4F480913E
:101D7000E800877F8093E8008091E7018093E0018D
:101D80000E94B00B8091E001811106C08091E300B8
:101D900087FD02C081E001C084E08093E4010E94DD
:101DA000FE088091E80083FF0AC08091E800877FE9
:101DB0008093E8008091EB0080628093EB00AA960C
:101DC0000FB6F894DEBF0FBECDBFDF91CF911F914C
:101DD00008950895CF938091E4018823A1F0C091E4
:101DE000E900CF709091EC00892F817090FD80E820
:101DF000C82B1092E9008091E80083FD0E94930DAA
:101E0000CF70C093E900CF910895909369018093BA
:101E100068010895E0916801F0916901309721F01F
:101E20000190F081E02D099480E00895E09168012F
:101E3000F0916901309721F00280F381E02D09943F
:101E40000895E0916801F0916901309721F00480D4
:101E5000F581E02D09940895209166013091670184
:101E60002817390771F09093670180936601E0911C
:101E70006801F0916901309721F00680F781E02D2B
:101E8000099408952091640130916501281739075C
:101E900071F09093650180936401E0916801F09185
:101EA0006901309721F00084F185E02D09940895AF
:101EB00008950C94580F0E94161B0E94C8040C949D
:101EC000DC1BCF92DF92EF92FF920F931F93CF9381
:101ED000DF93CDB7DEB72B970FB6F894DEBF0FBEFA
:101EE000CDBF0E94E0048BE6C82E81E0D82E00E032
:101EF00010E0E02E802F0E94D605F60141916F017F
:101F0000F82EF426B1F40F5F1F4F0E30110589F73C
:101F10008FEF89838A831B820E941F1B8160782F29
:101F20009D838C8349815A816B818D810E9404102D
:101F300040C09091CC0191FF04C08B870E94DC05CA
:101F40008B8520E030E04F2D50E0922FBA01022E19
:101F500002C0759567950A94E2F760FF24C02E834E
:101F6000EF8221E030E0690102C0CC0CDD1C9A95C3
:101F7000E2F790E08C219D21892B09F420E028874D
:101F80000E941F1B8160782F9A8789874E815F810D
:101F900068858A850E940410F801E559FE4F80810A
:101FA000C826C08206C02F5F3F4F2630310569F634
:101FB000AACF0E94C31E0E940A0F90916A0189173E
:101FC000A1F00E940A0F80936A012B960FB6F89435
:101FD000DEBF0FBECDBFDF91CF911F910F91FF905C
:101FE000EF90DF90CF900C9400082B960FB6F894EA
:101FF000DEBF0FBECDBFDF91CF911F910F91FF903C
:10200000EF90DF90CF900895CF93DF93CDB7DEB7F9
:102010002B970FB6F894DEBF0FBECDBF4F83588706
:1020200069877A878B87DE01119686E0FD01119220
:102030008A95E9F785E0FE01379601900D928A9521
:10204000E1F749815A816B817C818D819E810E945B
:1020500007172B960FB6F894DEBF0FBECDBFDF91EA
:10206000CF910895CF93C82F882309F4C1C0823837
:1020700059F40E940A0F81FDBBC089E30E94A41994
:102080000E945C1A89E30CC0833879F40E940A0F1D
:1020900080FDAEC083E50E94A4190E945C1A83E50E
:1020A0000E94E319CF910C945C1A843859F40E9471
:1020B0000A0F82FD9DC087E40E94A4190E945C1A49
:1020C00087E4EECF8CEF8C0F813A48F48C2F0E947E
:1020D000032181118DC08C2F0E94A419E3CF80E2CF
:1020E0008C0F883048F4C77081E001C0880FCA9512
:1020F000EAF70E94251AD6CF8BE58C0F833078F44F
:10210000C53A29F0C63A31F083E890E005C081E88D
:1021100090E002C082E890E0CF910C942C0F88E50B
:102120008C0F833108F064C0C83A39F1C93A41F1E3
:10213000CA3A49F1CB3A51F1CC3A59F1CD3A61F171
:10214000C03B69F1CE3A71F1CF3A79F1C13B81F1EF
:10215000C23B89F1C33B91F1C43B99F1C53BA1F16D
:10216000C63BA9F1C73BB1F1C83BB9F1C93BC1F1CD
:10217000CA3BC9F180E090E038C082EE90E035C003
:1021800089EE90E032C08AEE90E02FC085EB90E0BF
:102190002CC086EB90E029C087EB90E026C08CEC49
:1021A00090E023C08DEC90E020C083E891E01DC05A
:1021B0008AE891E01AC082E991E017C084E991E0D1
:1021C00014C081E292E011C083E292E00EC084E28A
:1021D00092E00BC085E292E008C086E292E005C082
:1021E00087E292E002C08AE292E0CF910C94420F23
:1021F000CF910895882309F44BC0823859F40E9486
:102200000A0F81FF45C089E30E94A4190E945C1A4D
:1022100089E30CC0833871F40E940A0F80FF38C034
:1022200083E50E94A4190E945C1A83E50E94E319C9
:102230000C945C1A843859F40E940A0F82FF28C05B
:1022400087E40E94A4190E945C1A87E4EFCF9CEFF8
:10225000980F913A58F390E2980F983050F48770A5
:1022600091E001C0990F8A95EAF7892F0E942B1AF5
:10227000DFCF9BE5980F933020F480E090E00C9442
:102280002C0F885A833120F480E090E00C94420FA8
:102290000895882321F00E94251A0C945C1A089551
:1022A000882321F00E942B1A0C945C1A0895BF9287
:1022B000CF92DF92EF92FF920F931F93CF93DF9312
:1022C00000D000D000D0CDB7DEB77C0185E0F701AB
:1022D000DE01119601900D928A95E1F7F701838155
:1022E0009481892B09F4DDC2908181818F3F19F49B
:1022F0009F3F09F4D6C2F7010281258122952F70F4
:1023000099838A8389819A812E830E946319182F69
:10231000B92E0E9462190E942918EB2DE295EF70E8
:102320004E2F50E0FA01E05AFF4F2E810C944723C4
:102330008B2D807F9B2D9F70F92E882319F0F294AE
:1023400080EFF822002349F0FF2009F457C28F2DB7
:102350000E94351A0E945C1A51C2812F0E94FA1005
:10236000FF2009F49EC28F2D0E943B1A26960FB6BD
:10237000F894DEBF0FBECDBFDF91CF911F910F91BB
:10238000FF90EF90DF90CF90BF900C945C1A3B2DA4
:10239000307F8B2D8F70303211F08295807F11232A
:1023A00019F0113021F12CC00023B9F0222309F4D7
:1023B00090C1213009F08DC126960FB6F894DEBF8A
:1023C0000FBECDBFDF91CF911F910F91FF90EF9086
:1023D000DF90CF90BF900C94451A222319F0213042
:1023E00009F45FC28E830E94481A8E8186C1002341
:1023F00021F0223008F055C26CC1211152C27DC1BA
:10240000002321F0222309F464C1F8C1222309F436
:1024100074C109C28B2D86958695837019F0813021
:10242000D1F03FC2002321F0812F9B2D937002C079
:1024300080E090E026960FB6F894DEBF0FBECDBFC9
:10244000DF91CF911F910F91FF90EF90DF90CF9090
:10245000BF900C942C0F002321F0812F9B2D9370A3
:1024600002C080E090E026960FB6F894DEBF0FBE63
:10247000CDBFDF91CF911F910F91FF90EF90DF9033
:10248000CF90BF900C94420F812F002319F00E942F
:10249000CB1D02C00E94331E26960FB6F894DEBFF5
:1024A0000FBECDBFDF91CF911F910F91FF90EF90A5
:1024B000DF90CF90BF900C94B81E8B2D837009F0E5
:1024C00075C00111EEC1812F829586958770880FA6
:1024D000880F912F9F70C92ED12CE12CF12C082E42
:1024E00004C0CC0CDD1CEE1CFF1C0A94D2F714FFB8
:1024F00012C00FE010E020E030E004C0000F111F18
:10250000221F331F8A95D2F7C901B80160957095D3
:102510008095909503C060E070E0CB014B2D46950F
:10252000469543704230C1F060F56C297D298E29B3
:102530009F29413051F126960FB6F894DEBF0FBEA9
:10254000CDBFDF91CF911F910F91FF90EF90DF9062
:10255000CF90BF900C9450186C297D298E299F290B
:1025600026960FB6F894DEBF0FBECDBFDF91CF9198
:102570001F910F91FF90EF90DF90CF90BF900C9440
:102580006C180E945018C701B60126960FB6F89431
:10259000DEBF0FBECDBFDF91CF911F910F91FF9096
:1025A000EF90DF90CF90BF900C943418002319F077
:1025B0008B2D817001C08695882309F472C1812F0B
:1025C000829586958770880F880F912F9F70C92EEE
:1025D000D12CE12CF12C082E04C0CC0CDD1CEE1CFF
:1025E000FF1C0A94D2F714FF12C00FE010E020E0A5
:1025F00030E004C0000F111F221F331F8A95D2F74D
:10260000C901B801609570958095909503C060E010
:1026100070E0CB014B2D4695469543704230C1F09A
:1026200060F56C297D298E299F29413051F126962C
:102630000FB6F894DEBF0FBECDBFDF91CF911F91D3
:102640000F91FF90EF90DF90CF90BF900C942A19DC
:102650006C297D298E299F2926960FB6F894DEBF16
:102660000FBECDBFDF91CF911F910F91FF90EF90E3
:10267000DF90CF90BF900C9446190E942A19C70191
:10268000B60126960FB6F894DEBF0FBECDBFDF9120
:10269000CF911F910F91FF90EF90DF90CF90BF905F
:1026A0000C940E19103FD1F118F4103E50F4A1C053
:1026B000123F09F463C008F44CC0133F09F473C01F
:1026C00098C01F708B2D8F710023A1F00E94A71856
:1026D000812F26960FB6F894DEBF0FBECDBFDF91D7
:1026E000CF911F910F91FF90EF90DF90CF90BF900F
:1026F0000C9449110E94C818812F26960FB6F894A1
:10270000DEBF0FBECDBFDF91CF911F910F91FF9024
:10271000EF90DF90CF90BF900C9450110023A9F060
:102720002111BFC08B2D8F7126960FB6F894DEBF96
:102730000FBECDBFDF91CF911F910F91FF90EF9012
:10274000DF90CF90BF900C94ED18223008F0A9C014
:10275000E9CF0023A9F08B2D8F7126960FB6F89440
:10276000DEBF0FBECDBFDF91CF911F910F91FF90C4
:10277000EF90DF90CF90BF900C94A718002359F3EF
:102780008B2D8F7126960FB6F894DEBF0FBECDBF8E
:10279000DF91CF911F910F91FF90EF90DF90CF903D
:1027A000BF900C94C818002399F08B2D8F7126963A
:1027B0000FB6F894DEBF0FBECDBFDF91CF911F9152
:1027C0000F91FF90EF90DF90CF90BF900C949218F4
:1027D00026960FB6F894DEBF0FBECDBFDF91CF9126
:1027E0001F910F91FF90EF90DF90CF90BF900C94CE
:1027F00088180023A9F0222309F4ADCF812F269653
:102800000FB6F894DEBF0FBECDBFDF91CF911F9101
:102810000F91FF90EF90DF90CF90BF900C9432100B
:10282000222309F4ADCF812F26960FB6F894DEBF90
:102830000FBECDBFDF91CF911F910F91FF90EF9011
:10284000DF90CF90BF900C94FA104B2D4F70612FFA
:10285000C7010E94360326960FB6F894DEBF0FBE5E
:10286000CDBFDF91CF911F910F91FF90EF90DF903F
:10287000CF90BF900C94AC174B2D4F70612FC701B8
:1028800026960FB6F894DEBF0FBECDBFDF91CF9175
:102890001F910F91FF90EF90DF90CF90BF900C941D
:1028A0009D0626960FB6F894DEBF0FBECDBFDF9112
:1028B000CF911F910F91FF90EF90DF90CF90BF903D
:1028C00008950E94421A0E94171A0E945C1A0E94E0
:1028D000681F0E94B81E80E090E00E942C0F80E0EC
:1028E00090E00C94420F0E94321A0C9461140E94E2
:1028F0006319292F22952F702C3030F42A3048F498
:102900002250223078F405C02C3041F02F3031F0C5
:1029100009C0803E48F0803F29F406C093FB882719
:1029200080F9089580E0089581E00895CF93DF93C2
:1029300000D000D01F92CDB7DEB70F900F900F9050
:102940000F900F90DF91CF910895CF93DF9300D038
:1029500000D000D0CDB7DEB726960FB6F894DEBF14
:102960000FBECDBFDF91CF9108951F93CF93DF931B
:10297000C091790116E080917A01C81799F0D0E0F2
:102980001C9FF0011D9FF00D1124E558FE4F408162
:10299000518162817381848195810E94A514219661
:1029A000C770E9CFDF91CF911F9108954091AB019E
:1029B0005091AC016091AD017091AE018091AF0179
:1029C0009091B0010C94A5148091B00182958F7004
:1029D00009F054C08091AD01882309F44FC0809163
:1029E0007901A0917A014091AE015091AF016091BF
:1029F000AB017091AC01B6E08A1709F43FC090E0DA
:102A000041155105C1F17F3F11F46F3FA1F1B89F0E
:102A1000F001B99FF00D1124E558FE4F21812713D5
:102A20002AC02081261327C02281211124C023819E
:102A300034812417350710F421503109241B350B3C
:102A4000283C3105C0F42091B0012F702061209303
:102A5000B00126E0289FF001299FF00D1124E058D5
:102A6000FE4F80818F70806180838BEA91E00E94AD
:102A700057110C94B51401968770BECF0895CF926C
:102A8000DF92EF92FF920F931F93CF93DF93CDB717
:102A9000DEB762970FB6F894DEBF0FBECDBF8C01D4
:102AA00085E0F801DE011D9601900D928A95E1F70F
:102AB000D8014C9111965C91119712966C9180916E
:102AC000AE019091AF01009709F475C13091AB014F
:102AD0007091AC017F3F19F43F3F09F46CC1F801DC
:102AE000C380D480E090AD01EE2009F4BEC02091F7
:102AF000B001C816D90628F0D601A81BB90BCD0124
:102B000004C0809590958C0D9D1DFF24F394883C06
:102B1000910578F0F12C207F09F0C4C07C2DD98A72
:102B2000C88A89890E9496148BEA91E00E94571105
:102B3000AFC0822F807F09F045C0571313C04313E5
:102B400011C061110FC02F7020612093B0010E944D
:102B5000D6148BEA91E00E9457118091B001F801E0
:102B600085832EC0CD2819F15F3F11F44F3FF9F056
:102B7000F62E61111CC08091790120917A0136E016
:102B8000821709F45BC090E0389FF001399FF00D87
:102B90001124E558FE4F7181571306C07081471309
:102BA00003C07281711103C001968770E9CFF62EC0
:102BB000662309F41CC18091B00181608093B0014B
:102BC000F12C15C1571309C0431307C0611105C08B
:102BD0008091B001F8018583C8C04D875E878D85DF
:102BE0009E856A8B0E9477146A898823D1F16623B7
:102BF000C1F12091B001822F82958F7090E00297F1
:102C000074F08091AB019091AC0198878F83198605
:102C1000DB86CA862C87CE0107960E94571186E074
:102C2000F801ABEAB1E001900D928A95E1F70E94BC
:102C3000E4140E94D614FF24F394D9C04D875E8714
:102C40008D859E850E946319292F22952F70223031
:102C500008F0C1C09F7009F0BBC0805E883008F4E6
:102C6000C6C0C8010E945711E6CFC816D90608F49D
:102C700053C0F601E81BF90BCF01883C910508F41D
:102C800050C0F12C7C2DD98AC88A89890E9496145B
:102C9000EBEAF1E086E0DF011D928A95E9F70E94F8
:102CA000D614A5C0571314C0431312C0611110C02D
:102CB0008091B001F8018583C8010E94571186E018
:102CC000EBEAF1E0DF011D928A95E9F7FE2C8FC057
:102CD0004D875E878D859E856A8B0E9477146A89F1
:102CE000882309F4BECF662309F4BBCF2091B0013D
:102CF000822F82958F7090E002970CF490CF809194
:102D0000AB019091AC019A8389831B82DD82CC82D6
:102D10002E83CE01019681CF809590958C0D9D1DBF
:102D2000ACCFF62E662309F49CCF571333C0431360
:102D300031C02091B00120FD24C0822F82958F7078
:102D4000482F50E041155105E1F0D80115962C931C
:102D500015974F30510549F08F5F982F9295907FCE
:102D6000822F8F70892B15968C93C8010E94571162
:102D700086E0F801ABEAB1E001900D928A95E1F7A7
:102D80008ECF86E0F801ABEAB1E001900D928A9512
:102D9000E1F72DC04D875E878D859E850E94771453
:102DA00081113DCF8091B00181608093B001C80155
:102DB0000E9457111CC0662309F453CF4D875E87CC
:102DC0008D859E850E947714882309F44ACF27CFEA
:102DD000811143CF0CC0243008F043CF9F7009F419
:102DE0003CCFD80115969C91907F09F036CF8F2D5E
:102DF00062960FB6F894DEBF0FBECDBFDF91CF91C4
:102E00001F910F91FF90EF90DF90CF9008951F9347
:102E1000CF93DF93CDB7DEB72C970FB6F894DEBF14
:102E20000FBECDBF4F83588769877A878B879C8772
:102E3000CE0107960E943F15882371F08A859B85F5
:102E4000892B09F441C088858F3F09F065C08F81C7
:102E50008F3F09F061C038C086E0FE013796DE0181
:102E6000119601900D928A95E1F76A857B8561152F
:102E7000710551F1FF81E885EF3F11F4FF3F21F12A
:102E800020917A0130E0C90101968770992740911D
:102E9000790150E08417950709F447C0F983EA8364
:102EA0007D836C8396E0929FD001939FB00D112497
:102EB000A558BE4FFE01319601900D929A95E1F70B
:102EC00080937A010E94B51416E080917901909167
:102ED0007A018917B9F1189FC001112485589E4FB6
:102EE0000E943F15882371F1E09179011E9FF00146
:102EF0001124E558FE4F40815181628173818481A4
:102F000095810E94A5148091790190E001968770C7
:102F1000992780937901D9CF4F81588569857A8522
:102F20008B859C850E94A514CFCF0E9473141092AC
:102F30007A0110927901EBEAF1E086E0DF011D925F
:102F40008A95E9F72C960FB6F894DEBF0FBECDBF79
:102F5000DF91CF911F910895EF92FF920F931F93EE
:102F6000CF93DF938C01892B09F46CC0F12CEE24F4
:102F7000E394E8012196F8018491843740F4843089
:102F800008F051C0813081F0823019F15BC0853783
:102F900009F444C0A8F19CE7980F903708F052C09C
:102FA0008F770E94FA1041C00E5F1F4FFE0184917F
:102FB00090E2980F983050F48770FE2D01C0FF0FFB
:102FC0008A95EAF78F2F0E94351A14C00E9432109A
:102FD0002DC00E5F1F4FFE01849190E2980F983034
:102FE00060F48770FE2D01C0FF0F8A95EAF78F2FDE
:102FF0000E943B1A0E945C1A19C00E94FA1016C067
:103000000E5F1F4FFE01C491CC2381F08FE99FE03A
:103010000197F1F700C00000C150F6CF0E5F1F4FBF
:10302000FE01F49003C00E9432108E018F2D882380
:1030300009F49FCFEFE9FFE03197F1F700C00000FE
:103040008150F5CFDF91CF911F910F91FF90EF90BD
:10305000089508956093B5017093B6018093B70108
:103060009093B8010C9461140F931F930091B501D4
:103070001091B6012091B7013091B801DC01CB016C
:10308000802B912BA22BB32B8093B5019093B6018B
:10309000A093B701B093B8011F910F910C946114E4
:1030A0000F931F930091B5011091B6012091B701C4
:1030B0003091B801DC01CB0180239123A223B323FB
:1030C0008093B5019093B601A093B701B093B80176
:1030D0001F910F910C9461140F931F930091B501F0
:1030E0001091B6012091B7013091B801DC01CB01FC
:1030F00080279127A227B3278093B5019093B6012B
:10310000A093B701B093B8011F910F910C94611473
:103110001092B1011092B2011092B3011092B40159
:103120000C94611441E050E060E070E004C0440F92
:10313000551F661F771F8A95D2F74093B1015093B0
:10314000B2016093B3017093B4010C94611441E037
:1031500050E060E070E004C0440F551F661F771F09
:103160008A95D2F78091B1019091B201A091B301FB
:10317000B091B401482B592B6A2B7B2B4093B101A2
:103180005093B2016093B3017093B4010C94611435
:1031900041E050E060E070E004C0440F551F661F3E
:1031A000771F8A95D2F740955095609570958091DC
:1031B000B1019091B201A091B301B091B401482343
:1031C00059236A237B234093B1015093B20160934A
:1031D000B3017093B4010C94611441E050E060E0DD
:1031E00070E004C0440F551F661F771F8A95D2F701
:1031F0008091B1019091B201A091B301B091B4015D
:10320000482759276A277B274093B1015093B20181
:103210006093B3017093B4010C9461140F931F93E6
:103220000091B1011091B2012091B3013091B4012C
:10323000DC01CB01802B912BA22BB32B8093B1010E
:103240009093B201A093B301B093B4011F910F9179
:103250000C9461140F931F930091B1011091B2016E
:103260002091B3013091B401DC01CB018023912383
:10327000A223B3238093B1019093B201A093B30131
:10328000B093B4011F910F910C9461140F931F938D
:103290000091B1011091B2012091B3013091B401BC
:1032A000DC01CB0180279127A227B3278093B101AE
:1032B0009093B201A093B301B093B4011F910F9109
:1032C0000C9461140895CF92DF92EF92FF920F93C6
:1032D0001F93CF93DF938C01C090B101D090B201C6
:1032E000E090B301F090B4018091B5019091B601E6
:1032F000A091B701B091B801C82AD92AEA2AFB2ABD
:10330000CFE1D0E0D701C6010C2E04C0B695A79539
:10331000979587950A94D2F780FF07C0B8018C2F44
:103320000E94C1068130910531F4219758F7B80108
:1033300080E00E94C106DF91CF911F910F91FF9015
:10334000EF90DF90CF90089590910C019923F1F0C8
:1033500090910D019923D1F0982F96959695969579
:103360009F3080F5E0910E01F0910F01E90FF11D02
:10337000877021E030E0A90102C0440F551F8A95F3
:10338000E2F7CA019181892B8183089520910E0172
:1033900030910F01F90132969FEF40E0519185176E
:1033A00089F09F3F19F4511101C0942F4F5F4E30A7
:1033B000A9F79F3F39F0F901E90FF11D97FDFA9543
:1033C00082830895089590910C019923F9F09091CA
:1033D0000D019923D9F0982F9695969596959F3043
:1033E00028F5E0910E01F0910F01E90FF11D8770B2
:1033F00021E030E0A90102C0440F551F8A95E2F791
:10340000CA018095918189238183089520910E01BD
:1034100030910F01F9013296205F3F4F908189135F
:1034200001C010823196E217F307C1F7089581E0D9
:1034300090E0E0910E01F0910F01E80FF91F10826A
:10344000019680319105A9F708959091CB01892BC0
:103450008093CB01089580959091CB01892380932F
:10346000CB0108951092CB0108959091CA01892B48
:103470008093CA01089580959091CA018923809311
:10348000CA0108951092CA0108958093B901089560
:103490001092B901089580910E0190910F01FC01E5
:1034A00031969C01205F3F4F80E0919191118F5F99
:1034B000E217F307D1F70895E0910E01F0910F01A3
:1034C0008091CB018083E0910E01F0910F019081FA
:1034D0008091CA01892B80838091B901882361F092
:1034E000E0910E01F0910F019081892B80830E9461
:1034F0004B1A81111092B90180910E0190910F0128
:103500000C94160FCF92DF92EF92FF926C01EE2493
:10351000FF24C114D104E104F10421F0C701B60174
:1035200020E101C020E0C72ED82EE92EFF24C114CF
:10353000D104E104F10419F0285FC701B6016B0161
:103540007C0154E0F694E794D794C7945A95D1F748
:10355000C114D104E104F10419F02C5FC701B601D4
:103560006B017C0142E0F694E794D794C7944A95A6
:10357000D1F7C114D104E104F10419F02E5FC701A1
:10358000B601DC01CB01B695A79597958795892B58
:103590008A2B8B2B09F02F5F822FFF90EF90DF900B
:1035A000CF9008958091E401843011F120E488E106
:1035B00090E00FB6F894A895809360000FBE20931A
:1035C000600083B7817F846083BF83B7816083BFDE
:1035D0007894889583B78E7F83BF0FB6F894A895AB
:1035E00080916000886180936000109260000FBE3F
:1035F000089508950C94F91ACF930E94FA1A0E9424
:10360000E0040E94F91AC0E08C2F0E94D6058111B7
:1036100004C0CF5FCE30C1F701C081E0CF910895E3
:103620000E9473140E940A0F0C94000882E084BD6B
:1036300093E095BD9AEF97BD80936E0008952FB7E4
:10364000F8948091CD019091CE01A091CF01B091DD
:10365000D0012FBF0895CF92DF92EF92FF920F9388
:103660001F932FB7F8944091CD015091CE016091F6
:10367000CF017091D0012FBF6A017B01EE24FF249E
:103680008C0120E030E0C016D106E206F30610F40B
:10369000415051099A01281B390BC9011F910F9103
:1036A000FF90EF90DF90CF9008951F920F920FB68A
:1036B0000F9211248F939F93AF93BF938091CD016D
:1036C0009091CE01A091CF01B091D0010196A11DA2
:1036D000B11D8093CD019093CE01A093CF01B09303
:1036E000D001BF91AF919F918F910F900FBE0F901E
:1036F0001F9018950E94020CF8942FEF87EA91E62C
:10370000215080409040E1F700C0000087E090EB3E
:10371000DC018093ED019093EE01A093EF01B09353
:10372000F0019CE088E10FB6F894A89580936000C2
:103730000FBE90936000FFCFEF92FF920F931F9305
:10374000CF93DF93D82FC0E08C2F0E94D60500E0E6
:1037500010E0E82EF12CC701002E02C09595879548
:103760000A94E2F780FD06C00F5F1F4F0630110577
:1037700091F709C0602F7C2F80E00E949E068D1378
:10378000F3CF81E004C0CF5FCE30F1F680E0DF916F
:10379000CF911F910F91FF90EF900895CF93C82F75
:1037A0008CE20E949C1B882321F08C2FCF910C94DB
:1037B0009C1B80E0CF910895CF930E94231D81111F
:1037C00002C00E94091DC5E6C15049F00E94E004F4
:1037D0008FE39CE90197F1F700C00000F5CF89E283
:1037E0000E94CE1B811113C18AE20E94CE1B81115F
:1037F0000E94091D85E00E94CE1B81110E947A1B48
:103800000E942E1D8093CC0187E00E94CE1B88234E
:10381000A9F18BE10E94CE1B882351F08091CC014D
:1038200081FB222720F991E0922790FB81F90EC0BD
:103830008EE00E94CE1B882361F08091CC0182FB38
:10384000222720F991E0922790FB82F98093CC0106
:1038500015C080E10E94CE1B9091CC01882341F0DD
:1038600093FB222720F981E0822780FB93F904C093
:10387000892F809580FB90F99093CC018091CC01A9
:103880000E94321D0E94401D8093DE0180EE0E9446
:10389000CE1B882341F08091DE01982F909590FBFC
:1038A00080F98093DE0189E30E94CE1B882359F0C2
:1038B0008091DE0181FB222720F991E0922790FB85
:1038C00081F98093DE0182EE0E94CE1B882359F09D
:1038D0008091DE0182FB222720F991E0922790FB64
:1038E00082F98093DE0186EE0E94CE1B882359F078
:1038F0008091DE0183FB222720F991E0922790FB43
:1039000083F98093DE0183EE0E94CE1B882359F059
:103910008091DE0184FB222720F991E0922790FB21
:1039200084F98093DE0185E30E94CE1B882359F041
:103930008091DE0185FB222720F991E0922790FB00
:1039400085F98093DE0181E30E94CE1B882359F024
:103950008091DE0186FB222720F991E0922790FBDF
:1039600086F98093DE0181E10E94CE1B882359F005
:103970008091DE0187FB222720F991E0922790FBBE
:1039800087F98093DE018091DE010E94441D8091C1
:10399000DE0187FB882780F980930D0187E20E9472
:1039A000CE1BC82F8EE10E94CE1B8111C2608FE119
:1039B0000E94CE1B8111C46080E20E94CE1B811147
:1039C000C86081E20E94CE1B8111C06182E20E9428
:1039D000CE1B8111C06283E20E94CE1B8111C064A4
:1039E00084E20E94CE1B882311F0C06802C0CC2361
:1039F00029F08C2F0E943B1D6C2F03C00E94371DA5
:103A0000682F70E080E090E0CF910C942A18CF915D
:103A100008956DEE7EEF80E090E00E947D2360E0EF
:103A200082E090E00E946F2360E083E090E00E94DB
:103A30006F2360E084E090E00E946F2360E085E007
:103A400090E00C946F2380E090E00E94692321E0D5
:103A50008D3E9E4F09F020E0822F089582E090E095
:103A60000C946123682F82E090E00C946F2383E034
:103A700090E00C946123682F83E090E00C946F2316
:103A800084E090E00C946123682F84E090E00C9433
:103A90006F238091D30180FF0BC06091130185E0FB
:103AA000689FB001112475956795759567952BC032
:103AB00081FF09C06091130185E0689FB001112466
:103AC0007595679520C082FF07C06091130185E05E
:103AD000689FB001112417C09091D4019923D1F0AF
:103AE00060911201961788F72091130185E0289FB5
:103AF00090011124929FA001939F500D112470E01A
:103B0000CA010E9433236038710540F461157105C4
:103B100019F406C065E070E0862F08958FE70895D8
:103B200081E008958091D30180FF08C06091110168
:103B300070E0759567957595679521C081FF06C002
:103B40006091110170E07595679519C082FF04C0FE
:103B50006091110170E010C09091D401992399F007
:103B6000609110019617A0F780911101899FC00103
:103B7000112470E00E9433236038710540F4611510
:103B8000710519F406C061E070E0862F08958FE793
:103B9000089581E00895803F21F40E94491D819598
:103BA00004C0813F29F40E94491D8093D7010895E4
:103BB000823F21F40E94491D819504C0833F29F46E
:103BC0000E94491D8093D6010895893F19F40E94EF
:103BD000921D05C08A3F31F40E94921D8195809309
:103BE000D80108958B3F21F40E94921D819504C055
:103BF0008C3F29F40E94921D8093D9010895843F3F
:103C000021F48091D501816017C0853F21F4809116
:103C1000D501826011C0863F21F48091D501846076
:103C20000BC0873F21F48091D501886005C0883F93
:103C300031F48091D50180618093D50108958D3F45
:103C400021F48091D30181600BC08E3F21F48091DB
:103C5000D301826005C08F3F29F48091D301846035
:103C60008093D3010895803F39F48091D70187FF75
:103C70006CC01092D70169C0813F29F48091D701AF
:103C80001816BCF362C09091D601823F29F497FFC9
:103C90005CC01092D60159C0833F19F41916CCF3B9
:103CA00054C0893F41F48091D80118160CF04DC0E2
:103CB0001092D8014AC08A3F29F48091D80187FF29
:103CC00044C0F6CF8B3F39F48091D90187FF3DC0C6
:103CD0001092D9013AC08C3F29F48091D90118166D
:103CE000BCF333C0843F21F48091D5018E7F17C08F
:103CF000853F21F48091D5018D7F11C0863F21F44D
:103D00008091D5018B7F0BC0873F21F48091D50135
:103D1000877F05C0883F31F48091D5018F7E8093E5
:103D2000D50113C08D3F21F48091D3018E7F0BC04C
:103D30008E3F21F48091D3018D7F05C08F3F29F400
:103D40008091D3018B7F8093D3018091D601811123
:103D50000EC08091D70181110AC08091D8018111D4
:103D600006C08091D901811102C01092D40108953A
:103D700085ED91E00E94210F0E941F1B9093D201BC
:103D80008093D10108951F93CF93DF938091D10148
:103D90009091D2010E942B1BAC019091D4019923E8
:103DA00021F02091140130E006C0209115018AE035
:103DB000289F900111244217530708F485C0809171
:103DC000D601C091D701D091D8011091D9018111AC
:103DD00007C0C11175C0D11173C0111171C074C079
:103DE0009F3F19F09F5F9093D401181624F40E940E
:103DF000491D8093D6018091D60187FF05C00E949E
:103E0000491D81958093D6011C1624F40E94491DFA
:103E10008093D7018091D70187FF05C00E94491D7B
:103E200081958093D7016091D601662331F1C091CD
:103E3000D701CC2311F1062E000C770B880B990BC0
:103E40000E943A2223E333E343E35FE30E949E228E
:103E50000E9402226093D6016C2FCC0F770B880B47
:103E6000990B0E943A2223E333E343E35FE30E948A
:103E70009E220E9402226093D7011D1624F40E9404
:103E8000921D8093D8018091D80187FF05C00E94C0
:103E9000921D81958093D801111624F40E94921DE1
:103EA0008093D9018091D90187FF05C00E94921D9E
:103EB00081958093D901DF91CF911F910C94B81E09
:103EC0009F3F09F08FCFA0CFDF91CF911F91089531
:103ED000E5EDF1E085E0DF011D928A95E9F71092AA
:103EE000D4011092D3010895833081F128F48130F8
:103EF00059F08230D1F00895853009F449C0B8F105
:103F0000863009F456C0089580911501262F30E0BF
:103F1000280F311D2F3F310524F4680F60931501E0
:103F200008958FEF80931501089580911401262F35
:103F300030E0280F311D2F3F310524F4680F6093C6
:103F4000140108958FEF8093140108958091130157
:103F5000262F30E0280F311D2F3F310524F4680F44
:103F60006093130108958FEF80931301089580915A
:103F70001201262F30E0280F311D2F3F310524F488
:103F8000680F6093120108958FEF809312010895D6
:103F900080911101262F30E0280F311D2F3F310570
:103FA00024F4680F6093110108958FEF809311013D
:103FB000089580911001262F30E0280F311D2F3FEA
:103FC000310524F4680F6093100108958FEF8093FA
:103FD00010010895833011F128F4813049F08230C6
:103FE00091F00895853081F120F18630C1F1089576
:103FF00080911501681720F4861B809315010895A0
:1040000010921501089580911401681720F4861B01
:104010008093140108951092140108958091130162
:10402000681720F4861B80931301089510921301E2
:10403000089580911201681720F4861B8093120165
:10404000089510921201089580911101681720F4CB
:10405000861B80931101089510921101089580919B
:104060001001681720F4861B8093100108951092A8
:10407000100108950F931F938D3109F46BC008F060
:104080003FC08E3009F47DC0C0F4873009F46EC0A3
:1040900068F4863009F0AFC08091CC01817F8E7FBB
:1040A0008093CC0181E08093DB01A6C0883009F4C5
:1040B00058C08B3009F49BC09EC0863109F497C06C
:1040C00078F4803109F470C0813109F094C00E9405
:1040D000731490910D0181E0892780930D0187C0B1
:1040E000893109F484C08B3109F085C08091CC01FD
:1040F00081FB222720F991E0922790FB81F94AC0A9
:10410000853309F45BC048F4873209F457C008F4DA
:104110005AC0893209F452C06EC0833438F48A33ED
:1041200008F067C0883309F462C065C0833409F4BD
:1041300045C0883409F05FC00E9473140FEF13ED7F
:1041400020E3015010402040E1F700C000000E9431
:104150007A1B4DC00E94BC210E940A0F0E940008D9
:1041600046C00E942E1D0E94401D41C09091CC016E
:10417000892F817090FF12C0917F9E7F9093CC0118
:104180003BC08091CC0182FB222720F991E092274D
:1041900090FB82F98093CC01992349F18091CC0165
:1041A00081608093CC0123C08091CC0183FB2227C6
:1041B00020F991E0922790FB83F9ECCF61E070E069
:1041C00080E090E010C08D5141E050E060E070E090
:1041D0008A019B0104C0000F111F221F331F8A9503
:1041E000D2F7C901B8010E942A180E94731481E015
:1041F00003C08953E9CF80E01F910F91089580E0BB
:1042000008950C94FF20CF93C82F8091DB0181305B
:1042100079F018F08230E9F187C0E0910E01F09159
:104220000F018081813169F0823209F07FC009C0BD
:10423000E0910E01F0910F018081813111F0823205
:1042400061F48C2F0E940121811104C08C2F0E94E7
:104250003A201DC081E090E01AC08C2F0E94FF2000
:10426000811114C0C43179F048F4CB3079F0C031F9
:1042700009F060C082E08093DB0108C0C93219F008
:10428000C83321F057C01092DB0154C081E0817027
:1042900053C0C93289F118F5C43171F1A8F4C7309F
:1042A00009F046C08AE08093150194E190931401CF
:1042B00093E0909313018093120188E080931101A1
:1042C00088E28093100134C0CE51C63088F5EC2FBF
:1042D000F0E0E65DFE4F80818093DA0129C0CE34A4
:1042E000E9F020F4CB3421F56AE013C0C13579F050
:1042F000C235F1F461E00DC08091DA01882319F034
:104300001092DA0115C081E08093DB0115C061E0F5
:1043100006C08091DA010E94741F0AC06AE0809191
:10432000DA010E94EA1F04C01092DB0180E004C0A1
:1043300081E002C080E0ABCFCF910895E1E8F0E0EA
:104340008081886080838081816080838FB7F894CA
:1043500093E09093890090ED909388008FBF08952B
:10436000EFE6F0E08081826080830895EFE6F0E080
:1043700080818D7F80830895EFE6F0E0908182E078
:104380008927808308951F920F920FB60F921124F0
:104390002F933F934F935F936F937F938F939F934D
:1043A000AF93BF93EF93FF938091DC019091DD0178
:1043B00001969093DD018093DC01811103C082E0BE
:1043C0000E940008E091DD01E695E695F0E0E656F2
:1043D000FA4FE4918091DC018E1303C080E00E94CB
:1043E0000008FF91EF91BF91AF919F918F917F91C5
:1043F0006F915F914F913F912F910F900FBE0F9052
:104400001F9018950E9409226894B1110C9498226B
:1044100008950E947D2288F09F5798F0B92F992720
:10442000B751B0F0E1F0660F771F881F991F1AF09F
:10443000BA95C9F714C0B13091F00E949722B1E04B
:1044400008950C949722672F782F8827B85F39F04A
:10445000B93FCCF3869577956795B395D9F73EF438
:1044600090958095709561957F4F8F4F9F4F0895E0
:10447000E89409C097FB3EF49095809570956195FE
:104480007F4F8F4F9F4F9923A9F0F92F96E9BB27B4
:104490009395F695879577956795B795F111F8CF30
:1044A000FAF4BB0F11F460FF1BC06F5F7F4F8F4F9B
:1044B0009F4F16C0882311F096E911C0772321F091
:1044C0009EE8872F762F05C0662371F096E8862F29
:1044D00070E060E02AF09A95660F771F881FDAF780
:1044E000880F9695879597F9089557FD9058440F32
:1044F000551F59F05F3F71F04795880F97FB991F43
:1045000061F09F3F79F087950895121613061406FF
:10451000551FF2CF4695F1DF08C01616170618068C
:10452000991FF1CF86957105610508940895E89467
:10453000BB2766277727CB0197F908950E94B12200
:104540000C9422230E94142338F00E941B2320F095
:10455000952311F00C940B230C94112311240C942B
:1045600098220E94752270F3959FC1F3950F50E039
:10457000551F629FF001729FBB27F00DB11D639F15
:10458000AA27F00DB11DAA1F649F6627B00DA11DBB
:10459000661F829F2227B00DA11D621F739FB00D61
:1045A000A11D621F839FA00D611D221F749F3327D1
:1045B000A00D611D231F849F600D211D822F762F6A
:1045C0006A2F11249F5750409AF0F1F088234AF047
:1045D000EE0FFF1FBB1F661F771F881F91505040B3
:1045E000A9F79E3F510580F00C940B230C94982260
:1045F0005F3FE4F3983ED4F3869577956795B7953A
:10460000F795E7959F5FC1F7FE2B880F911D969553
:10461000879597F9089597F99F6780E870E060E0C3
:1046200008959FEF80EC089500240A94161617064B
:1046300018060906089500240A9412161306140693
:1046400005060895092E0394000C11F4882352F0F6
:10465000BB0F40F4BF2B11F460FF04C06F5F7F4FAE
:104660008F4F9F4F089597FB072E16F4009407D0A5
:1046700077FD09D00E944D2307FC05D03EF49095AC
:1046800081959F4F0895709561957F4F0895EE0F26
:10469000FF1F0590F491E02D0994AA1BBB1B51E16B
:1046A00007C0AA1FBB1FA617B70710F0A61BB70BA2
:1046B000881F991F5A95A9F780959095BC01CD0147
:1046C0000895F999FECF92BD81BDF89A992780B5DA
:1046D0000895A8E1B0E042E050E00C948423262F36
:1046E000F999FECF1FBA92BD81BD20BD0FB6F894D7
:1046F000FA9AF99A0FBE019608950E946F23272F08
:104700000C947023DC01CB01FC01F999FECF06C0AB
:10471000F2BDE1BDF89A319600B40D92415050407F
:08472000B8F70895F894FFCFEB
:104728002002010891086C08380804080101BA0140
:1047380028080A03140A3F4D36395B050E05D804CC
:104748009F0432044B0464047D040102030405063B
:044758000708090045
:00000001FF
